:030000000211EEFC
:03000B000200BE32
:03002B00020400CC
:03005B0002054457
:0300730002053A49
:1000800002030406080C10182030406080020304AC
:1000900006080C101820304080FF0406080C1018C9
:1000A0002030406080A0C000000001010003020277
:1000B000010505020D0505050D0604050202C2AF86
:1000C000C0D0C0E0205A25302F02E47330601A05FA
:1000D00060C37405952540F2956040EE758A78E519
:1000E000257003758A000203F90203EC306306D21F
:1000F00092D291D29085258AC25AE525F4700221C8
:10010000DF0561306013206A19758B00D0E0D0D014
:10011000D292D291D290D2AF32D292D291D29002D8
:1001200001CFD26EC26FE565601CC3E561149565B1
:100130004014C26ED26FC3E561956450030201CFD3
:100140007561000201CF206C14D292D291D29074CA
:1001500006D5E0FDD293D294D2950201CFD26FD2D0
:1001600092D291D290E53D20E23420E1127406D57E
:10017000E0FD207502D295307502D2930201CF20A6
:10018000E0127406D5E0FD207502D295307502D2DA
:10019000930201CF7406D5E0FDD2940201CF20E195
:1001A0001F20E00A7406D5E0FDD2940201CF740648
:1001B000D5E0FD207502D293307502D2950201CFB1
:1001C0007406D5E0FD207502D293307502D2957584
:1001D0008B00D0E0D0D0D292D291D290D2AF32D098
:1001E000E0D0D0D2AF3261ECE525600A207502C2C2
:1001F00092307502C290D29161ECE5256002C29105
:10020000207502D290307502D29261ECE525600A29
:10021000207502C290307502C292207502D29230CF
:100220007502D29061EC207502C293307502C295BE
:10023000E525600A207502C292307502C2902075D1
:1002400002C295307502C293D29161EC207502C250
:1002500093307502C295207502C295307502C29323
:100260007406D5E0FDE525600A207502C29230755E
:1002700002C290D29161EC207502C293307502C225
:1002800095E525600A207502C292307502C290C2BF
:1002900094D29161EC207502C293307502C295C26E
:1002A000947406D5E0FDE525600A207502C29230FF
:1002B0007502C290D29161ECC294E5256002C291B0
:1002C000207502C293307502C295207502D290301B
:1002D0007502D29261ECC294207502C2933075020D
:1002E000C2957406D5E0FDE5256002C29120750235
:1002F000D290307502D29261ECC294E5256002C2C0
:1003000091207502C295307502C293207502D29079
:10031000307502D29261ECC294207502C29530759C
:1003200002C2937406D5E0FDE5256002C2912075F6
:1003300002D290307502D29261EC207502C29530E3
:100340007502C293E525600A207502C290307502DD
:10035000C292C294207502D292307502D29061ECA2
:10036000207502C295307502C293C2947406D5E01E
:10037000FDE525600A207502C290307502C2922008
:100380007502D292307502D29061EC207502C2954E
:10039000307502C293E525600A207502C29030755F
:1003A00002C292207502C293307502C29520750276
:1003B000D292307502D29061EC207502C2953075F0
:1003C00002C293207502C293307502C2957406D59D
:1003D000E0FDE525600A207502C290307502C292E8
:1003E000207502D292307502D29061ECE525F4F5C9
:1003F0008A758B00756000D25AD0E0D0D0D2AF326F
:10040000C2AFC0D0C0E0D2D3C2CEE528600A741F0C
:10041000552E60491528815D78007900E580307699
:1004200001F430E40278FF53DACF20760343DA2078
:1004300030760343DA10C2D8C269E580307601F421
:1004400030E40279FFC3E89970CE3059037528185B
:10045000741F552E60037528188858D268E52960E6
:100460000415298170741F552E600543DA01C2D826
:0E047000206802A102E558F8C268741F552EDC
:10047E0060367982B70431C3E894F0400374F0F823
:10048E00E8C4540F28F87984B7030281B6C313C3A6
:10049E00138721200802C313200A06C3C898F881C7
:1004AE00B628F8500374FFF8C3E8955F5003E55F74
:1004BE00F8E52C5406703D882230630AC3E5229578
:1004CE005C4003855C227882B60429C3E52295241C
:1004DE00401278A096400DE52426F5245009752487
:1004EE00FF0204F5852224852425C3E524955C406E
:1004FE0003855C2520CF09D0E0D0D0C2D3D2AF3255
:10050E00C2CF7801E5286008741F552E7002152899
:10051E00C3E55894014005755B00A131E55B0460AD
:10052E0002055BD0E0D0D0C2D3D2AF32C2AF53916E
:10053E007FC258D2AF32C2AFC0D0C0E0C0F0D2D36B
:10054E00A8FBA9FCC2D8306902A1A753DACF207646
:10055E000343DA1030760343DA20D269E580307631
:10056E0001F420E402A17B88268927E14753DACFE4
:10057E0020760343DA2030760343DA10C2D8C269FC
:10058E00741F552E7002E12D7800E580307601F44F
:10059E0030E402E12D8858E12D53DACF2076034363
:1005AE00DA2030760343DA10C269205902C1615352
:1005BE00DACF20760343DA1030760343DA20C2D83E
:1005CE00D26988538954C3E89551F8E99552F9E4F4
:1005DE00FB7AFAC3E894C8E994005008E4D2E4FB2D
:1005EE007A0AC134C3E89468E994015008E4D2E36E
:1005FE00FB7A0FC134C3E894D0E994025008E4D2D8
:10060E00E2FB7A1EC134C3E894A0E994055008E4D5
:10061E00D2E1FB7A3CC134C3E89498E994085006C1
:10062E00E4D2E0FB7A78C3E89555FCE99556FD30A7
:10063E00E708ECF42401FCEDF4FD7557007008C3D7
:10064E00EC9A500375570188558956A853A95488BA
:10065E00518952C3E89526F8E99527F9307402E1DD
:10066E0000307302E100307202C1F9E9C313F9E8F8
:10067E0013F8307102C1F9E9C313F9E813F83070B9
:10068E0002C1F9E9C313FDE813FC205918C3EC9419
:10069E001CED9402400302072DED7009C3EC94C8C3
:1006AE00500302074774002077037896E624FAFE7B
:1006BE00E43400FFC3EC9EFCED9FFD5006780079FC
:1006CE0000E100C3EC94FFED9400400678FF790042
:1006DE00E100EC856CF0A4C5F0A2F733F879004088
:1006EE000302071C78FF790002071CE9C313F9E81F
:1006FE0013F830740EE9600278FFC3E81338F8E49B
:10070E003400F9C3E894FFE99400400278FF88585A
:10071E00D268205902E12D741FF4552E4BF52E751B
:10072E002818741F552E700375280A305902E14798
:10073E00741F552E600353DAFE752906741F552E4D
:10074E00700375290AD0F0D0E0D0D0C2D3D2AF3228
:10075E007901E1767903E176790AE176791EE1761F
:10076E007964E17679C8E1767817E4D5E0FDD8FAB8
:10077E00D9F6227A147B7802079D7A107B8C0207B9
:10078E009D7A0D7BB402079D7A0B7BC802079DAC48
:10079E00257525017902B275E4C294D5E0FDE525F3
:1007AE006002C291D5E0FDD291D5E0FDD294D5E0A4
:1007BE00FDE525600A207502C292307502C290E5F1
:1007CE006DD5E0FD207502D292307502D2907496EE
:1007DE00D5E0FDD9C1EAF8D5E0FDD8FBDBB1C29476
:1007EE008C2522C37C007D0075F00005F0EA33FAFB
:1007FE00EB33FB50F6EB13FBEA13FAC3E9FFE8FE0B
:10080E00E89AF8E99BF95004EFF9EEF8B3EC33FCF3
:10081E00ED33FDD5F0DFEDF9ECF822E889F08A2012
:10082E00D2D4F8A9F07B0030F70B7BFFF42401F84B
:10083E00E9F43400F9E88520F0A4ADF0F8E985205C
:10084E00F0A4AFF0FEED2EF974003FFA7C04C3EA7B
:10085E0013FAE913F9E813F8DCF48BF030F70AE831
:0F086E00F42401F8E9F43400F9E889F0C2D4F871
:10087D00A9F0227882B6040302090CC3E55894014D
:10088D004018E54870377805C37994B7020278129D
:10089D00C3E53B9400E53C984020E5486009855E42
:1008AD005D7562FF756301852224E4F53FF540F522
:1008BD0041F542F543F54802090C754801C3799499
:1008CD00E79402601BE523F43333F913F8E954017F
:1008DD0004F9E854FEC39440F8E99400F9020908BC
:1008ED00E523F433333333F913F8E954070404F9EA
:1008FD00E854F8C39440F8E99400F9883F89402200
:10090D00E548603BC3E53C13F9E53B13F8C3E53F10
:10091D0098F8E54099F9500CC3E89480E994FF40AC
:10092D0016020948C3E8947FE99400500302094870
:10093D00787F7900020948788079FF8844894522BB
:10094D00E5486058E5442541F8E5453542F98545CA
:10095D0020E4300701F43543FA30E709C3EA94F097
:10096D00401502098AC3EA940F500302098A78FFE1
:10097D0079FF7A0F02098A780079007AF0C3E524AD
:10098D00955C5006E524600921A3E54520E70D217E
:10099D00A3E54530E706884189428A4322E5487040
:1009AD0003020A0D789EE6FAC3E54433F8E54533B4
:1009BD00F91129E930E70BC3E89480E994FF40135E
:1009CD0021E4C3E8947FE99400500221E4787F7913
:1009DD000021E4788079FFE820E715C3E52398F836
:1009ED004009C3E894014003020A0B7801020A0B87
:1009FD00E8F424012523F84003020A0B78FF88460A
:100A0D0022E5487003020A6F789FE6FAA842A943CF
:100A1D001129E930E70CC3E89401E994FF4016026F
:100A2D000A46C3E894FFE994005003020A4678FF92
:100A3D007900020A46780179FFE920E715C3E546FA
:100A4D0098F84009C3E894014003020A6D7800024A
:100A5D000A6DE8F424012546F84003020A6D78FF7B
:100A6D00882422020B077883E6F520120F6A75E8B9
:100A7D0090E5E820ECEDA8BDA9BE120FFF7568AF9B
:100A8D00756900C3740013FD74AF13FC74AF2CFCB7
:100A9D0074003DFDECFAEDFBC3E89AE99B4014E5CB
:100AAD006824AFF568E5693400F569EA2CFAEB3D89
:100ABD00FB80E5AE68AF69C3E56913F9E56813F826
:100ACD00C3E913F9E813F8E56828F566E56939F522
:100ADD00677A03C3E913F9E813F8DAF7AA201A7055
:100AED0009756800756900020B071AEA6008EE289F
:100AFD00FEEF39FFDAF88E688F692275E89022785B
:100B0D0083E6FFE5E820ECF7A8BDA9BE056AC3E5BD
:100B1D006A94084052756A00E97007E56B601B0224
:100B2D000B3BC3E8956B6010E56B5006600C14022F
:100B3D000B470460F9020B47E56BF56BC39458F84E
:100B4D004021755CC0C3E89404F84017755C80C300
:100B5D00E89404F8400D755C40C3E89404F8400334
:100B6D00755C0075BB0322C3E56AB4070375BB1042
:100B7D002230610278323062027878E52C540660BA
:100B8D001FE879A187F0A4C5F0A2F733F8C3E89563
:100B9D005C4002A85C882288248825306102885E2A
:100BAD0022788FE6FFC3EF94055018C3EF940450DD
:100BBD0020C3EF94035028C3EF94025030C3EF9439
:100BCD000150387533A075340F75353C7536058178
:100BDD00167533C075341275354075360681167528
:100BED0033707534177535D0753607811675334CDE
:100BFD0075341D7535C475360981167533287534F0
:100C0D00237535B875360B811685334F8534507580
:100C1D003B00753C0822A84FA950020C2EA849A9EB
:100C2D004A759100C3E498F594E499F5957591048E
:100C3D00D25875C820A8CCA9CD75C824AA39AB3A0D
:100C4D008839893AC3E89AF8E99BF9AA3BAB3CC3CA
:100C5D00EB13FDEA13FCC3ED13FDEC13FCC3EA9C8F
:0E0C6D00FAEB9DFBEA28FAEB39FB8A3B8B3C45
:100C7B00400122753BFF753CFF2230580281857580
:100C8B009100C3E4954BF594E4954CF5957591045F
:100C9B00D258227892E6FF7E10305B027F053063DC
:100CAB00047F037E00A93CA83B7A04C3E913F9E84F
:100CBB0013F8DAF7C3E89EF8E99400F94009C3E8A2
:100CCB009402E9940050047802E4F9E9FBE8FAC3D2
:100CDB00E913FDE813FCC3EF9403602EEF20E00D46
:100CEB00E82CF8E93DF9ECFAEDFB020D02E828F8E7
:100CFB00E939F97A02E4FBC3EF9403400D8A4D8B7B
:100D0B004E8849894A8C4B8D4C22884D894E8A4995
:100D1B008B4A8C4B8D4C22305802A122759100C30B
:100D2B00E4953BF594E4953CF595759104D25822E6
:100D3B00753E00752000020D4A753E00752040D2AD
:100D4B00AF053E20580122759D00E53CC313C3132C
:100D5B00F8086030306A06C313C313F808C3E8946D
:100D6B000A4002780A306D08C3E894044002780404
:100D7B00C3E53C9408400D759D02C3E53C941040BF
:100D8B0003759D03205803D2AF22791E206D027983
:100D9B000AD2AF0000C2AF205A0A793C206D02790B
:100DAB0014306FE03063027978C3E58B99206302CE
:100DBB0040F740D0E59BF4F45440B52002A14AD84B
:100DCB00C3D2AF22C25B789CE6146007E53E147079
:100DDB0002D25B30630B0538205810753800020DBA
:100DEB00F62058071581158102174022759100C313
:100DFB00E4954DF594E4954EF595759104D25822F2
:100E0B00AE25305B4F78A3E6FFBF010BD25C752597
:100E1B0000D292D291D290918A305C03752500302A
:100E2B005802C124BF020BD25C752500D292D2911D
:100E3B00D29078A2B6010D918A305C0375250030F3
:100E4B005802C144BF030BD25C752500D292D291DC
:100E5B00D290B1F7305C03752500305802C15F307A
:100E6B005B04C25C8E2522C2AFC294206A03020EC1
:100E7B0091900360306E0F207502C295307502C2DF
:100E8B00937406D5E0FD207502D293307502D2958E
:100E9B00759F10753D02D2AF22C2AF206A03020EBE
:100EAB00C6900317306E17C294207502C295307529
:100EBB0002C2937406D5E0FD020EC99001FA2075AB
:100ECB0002D290307502D292305A06E5256002C2EA
:100EDB0091207503759F20307503759F00753D0339
:100EEB00D2AF22C2AF207502C293307502C29520D9
:100EFB006A03020F0D9002D6306E07C2947406D5AA
:100F0B00E0FD207502D295307502D29320750375E2
:100F1B009F00307503759F20753D04D2AF22C2AF81
:100F2B00206A03020F4B900295306E17207502C298
:100F3B0093307502C295C2947406D5E0FD020F4E34
:100F4B009001E8D291305A0EE525600A207502C255
:100F5B0092307502C290759F10753D05D2AF22C2BB
:100F6B00AF207502C295307502C293206A03020F3F
:100F7B009190024C306E0F207502C293307502C2F5
:100F8B00957406D5E0FDD294207503759F203075BE
:100F9B0003759F00753D06D2AF22C2AF206A0302D4
:100FAB000FCF9003B9306E1F207502C293307502BC
:100FBB00C295207502C295307502C2937406D5E0B6
:100FCB00FD020FD290020C207502D292307502D224
:100FDB0090305A0EE525600A207502C290307502DA
:100FEB00C292207503759F00307503759F20753D68
:100FFB0001D2AF229001E6D292D291D290C293C28B
:10100B0094C29522C3E54F9535E550953650012294
:10101B007890E6FFC3EF94055018C3EF9404501B70
:10102B00C3EF9403501EC3EF94025021C3EF9401FE
:10103B005024C3E54F943CF802106AC3E54F942843
:10104B00F802106AC3E54F941AF802106AC3E54F11
:10105B009412F802106AC3E54F940AF802106AE57D
:0F106B00509400F9884F895022305803021074B6
:10107A0022788476037885760478867609788F765E
:10108A0003789076057895760278927603789B763F
:10109A000D7893760578877604789C760178887639
:1010AA00017889760178827604788C7601788D7653
:1010BA0000788E76B478967625789776D078987672
:1010CA0078789976C8789A7604789D76002278930B
:1010DA00E6FF756409756501C3BF02097564057584
:1010EA00650102111DC3BF03097564057565020216
:1010FA00111DC3BF040975640575650302111DC37B
:10110A00BF0506756409756507C3BF0606756400E1
:10111A007565007887E6FFC26CC3BF0302D26CC252
:10112A006BC3BF0402D26BC26A7418552D6002D217
:10113A006AC26E6002D26ED26F6002C26FC27578E6
:10114A0088E630E102D275C2767889E630E102D2C9
:10115A0076C3EF94026008758E01D26D02116E7526
:10116A008E00C26D227880E61490008093789EF6F5
:10117A007881E61490008093789FF6120FFF227808
:10118A009BE61490008D9378A0F6120FFF227886C2
:10119A00E61490009A9378A1F6120FFF22789CE643
:1011AA00149000A79378A2F6789CE6149000AC936A
:1011BA0078A3F6120FFF22227896E6FA7897E6FBD2
:1011CA003077047A007BFFC3EB9AFCC39482500207
:1011DA007C82756C00056CEC856CF0A4C3E5F09418
:1011EA008040F222C2D353D9BF7581C043FF801217
:1011FA00075E75EF0243B203E5B324044002F5B378
:10120A007580FF75A40075F1D475D4EF7590877554
:10121A00A54075F2FF75D5BF75A60175E24275DB6B
:10122A004675EA02120FFFE4F8F6D8FD117B121791
:10123A007011D8316F3189319831A731C131C278F3
:10124A0098866D120FFF75885075890275C82475C6
:10125A00910475D84012077212078112076A1207A1
:10126A008812076A12078F12076A121CCD120772B8
:10127A0012077212076E75A82275B80275E6907584
:10128A00F610759B80759D0375D10E75BC5875BB9C
:10129A000375BA1175E88012075ED2AF120A70435D
:1012AA00DA01C2D8C269120772753001D2597A05B9
:1012BA00E55770027A05120762E558C3940240EEB8
:1012CA00E52E541F855A59F55AB559E2DAE2C25940
:1012DA0053DACF20760343DA2030760343DA10C29A
:1012EA00D8C26912076E1207627802741F552E70EF
:1012FA00027800C3E5589840EDC2AF120781120781
:10130A0081120781D2AF12077275470012076278FD
:10131A008CE6C3940150030213DFE530C3940150F5
:10132A00030213DF741F552E6035C3E55894FF502E
:10133A00030213DFC2AF120796D2AF12076EC3E5DC
:10134A0058940150EFC2AF12078112076612078143
:10135A00D2AF12076EC3E55894FF40E9021D527FCF
:10136A0005D27731C212076EC2AFC27731C2C3E566
:10137A0058947FD2AF4068C2AF120796D2AFDFE16E
:10138A00C3E55894057897F612077212180C121CC6
:10139A00D57F0AD27731C212076EC2AFC27731C285
:1013AA00C3E558947FD2AF50E8C2AF120781120743
:1013BA0066120781D2AFDFDBE55824057896F6126C
:1013CA00077212180C121D0412076EC3E55894FF17
:1013DA0040F6021D52C3E558954740038558471207
:1013EA00076EC3E558940140026116C2AF12079610
:1013FA00120796120796D2AF120772753000E4F5FB
:10140A0031F5320531E531F470360532789AE678ED
:10141A0028146012785014600D78A014600878F0CF
:10142A00146003753200C3E5329840141532789976
:10143A00866DC2AF120796D2AF7898866D12076E84
:10144A00120762E5287008741F552E700241B6C350
:10145A00E558940640AD12076EE52870030212B6ED
:0F146A00120FFFE4F522F523F524F525755CFF3D
:101479007885865FF53FF540F541F542F543F56A14
:10148900F548F52BF52CF55B120BAE756A0875BBA3
:101499001012075E120B08E5E820ECFBA8BDA9BEF7
:1014A900E97001F8886B120B0C756A0875BB107826
:1014B90095E630E0030214FD7887E6FE760211D83E
:1014C9007887EEF6D261C2AF120B7E85225C852247
:1014D9005DD2AFC261752500756200756301D26086
:1014E900D263753800120F6A120FA5120C2A120B5B
:1014F900AE0216267887E6FE76037893E6FD760532
:1015090011D87887EEF67893EDF6D260D261D26E73
:10151900120F6A120FA5120B7E12075E120E7212BB
:10152900075E12075E120EA4120762120EEE120770
:1015390062120762120F29120766120F6A120762F6
:1015490012075EC261D262120B08120B0C120B7EDB
:10155900756A0875BB10120FA5120C23120C9E1187
:101569000F1174120E72120C23120C9E110F1174AA
:10157900120EA4120C23120C9E110F1174120EEEEE
:10158900120C23120C9E110F1174120F29120C2325
:10159900120C9E110F1174120F6A120C23120C9E59
:1015A900110FC3E54F9535E5509536400C1174C3BD
:1015B900E558940150910217401174C2627887E688
:1015C900FE760211D87887EEF685225C855E5D8508
:1015D9005E25756200756301D263753800C2AF205C
:1015E9007502C293307502C295207502C295307595
:1015F90002C293742DD5E0FDD2AF120FA5120C2AA9
:10160900120C85120C9E120D22756A0075BB03021D
:10161900162611D8120FA5756A0075BB03120D4461
:10162900120DCF120DF7120880120E0B120E721244
:101639000C2A120C85120C9E120D22120D3B120D52
:10164900CF120DF712090D120E0B120EA4120C2A4D
:10165900120C85120C9E120D22120D44120DCF127E
:101669000DF712094D120E0B120EEE120C2A120C66
:1016790085120C9E120D22120D3B120DCF120DF781
:101689001209AA120E0B120F29120C2A120C85121A
:101699000C9E120D22120D44120DCF120DF7120AD3
:1016A9000E120E0B120F6A120C2A120C85120C9EC6
:1016B900120D22120D3B120B08120DCF120DF7124B
:1016C9000B0C120E0B120FA5120C2A120C85120C00
:1016D9009E120D2230632A755CFF755DFF756200ED
:1016E900756301C3E5389464400AC263D2647537EF
:1016F9001402170AC3E5589401400302162602177B
:1017090040306419E537147005C26402161BF537B9
:10171900C3E55894014003021626021740C3E55B4E
:1017290094825013741F552E7004E5286009C3E58F
:101739003C94F05002C126120FFF7887E6FE76022C
:1017490011D87887EEF6E4F522F523F524F525F589
:101759005FC26012075E120FFF741F552E7006E5F7
:1017690028700241B68108901A0D7820121C00E5F4
:1017790020B45A0CA3121C00E520B4A5030217914A
:10178900117B12180C02180B78827604901A0778CC
:1017990084121C00A308121C00A308121C00A30831
:1017A900121C00A308121C00A308121C00A308A302
:1017B90008A308121C00A308A308A308121C00A36D
:1017C90008121C00A308A308121C00A308121C007D
:1017D900A308A308121C00A308121C00A308121CCA
:1017E90000A308121C00A308121C00A308121C0065
:1017F900A308121C00A308121C00A308121C0090C5
:101809001A2122C2AF121C3F121C19901A00740A25
:10181900121C05A37404121C05A37410121C059054
:101829001A077884121C04A308121C04A308121CAA
:1018390004A308121C04A308121C04A308121C0404
:10184900A308A308A308121C04A308A308A3081249
:101859001C04A308121C04A308A308121C04A3084F
:0F186900121C04A308A308121C04A308121C04D9
:10187800A308121C04A308121C04A308121C04A326
:1018880008121C04A308121C04A308121C04A308B1
:0D189800121C04121C52121C30901A212246
:101A00000A0410FFFFFFFF0304090401015AA501A6
:101A1000FFFF0305FF0305FF0225D0FAFA040D01BD
:021A200000FFC5
:101A400023484B696E673530412320202020202019
:101A500023424C48454C4923463333302320202031
:101A60002020202020202020202020202020202076
:101C0000E493F622E6438F01538FFD75EF0275B71B
:101C1000A575B7F1F0538FFE22438F02438F0175F4
:101C2000EF0275B7A575B7F1901A0DF0538FFC222E
:101C3000901A0D745A9105901A0E74A59105227A86
:101C40003079D07820901A409100E520F709A3DA86
:101C5000F7227A3079D0901A40E7910509A3DAF992
:101C600022AB6EA86FBB01057984021CCABB0205BA
:101C70007985021CCABB03057995021CCABB040501
:101C80007986021CCABB0505798F021CCABB0605F2
:101C90007990021CCABB07057992021CCABB0805D1
:101CA000799B021CCABB09057993021CCABB0A05B1
:101CB0007987021CCABB0B05799C021CCABB0C05A8
:101CC0007988021CCA7989021CCAE8F7227C0512AD
:101CD0000772DCFB22C2AF12078112078812078F3E
:101CE00012079612076612078112078812078F12D1
:101CF000079612076612078112078812078F1207CC
:101D000096D2AF22C2AF12079612078F120788121F
:101D1000078112076612079612078F1207881207AB
:101D20008112076612079612078F12078812078121
:101D3000D2AF22AE6EAF6FC2AF120781120781120F
:101D40000781120766DEF2120796120766DFF8D2E5
:101D5000AF2291D591CD91CD756E01756F017570E2
:101D600000B1337C05AD58120772C3ED955870F57C
:101D7000C3E55894014009C3E55894FF4032A18E51
:101D8000916112180C91D5C2AF75EF1291CDDCD5CF
:101D90000570C3E5709403500280C691CD056FE5D0
:101DA0006E149000B193F808C3E56F98500280AEAE
:101DB00091CD91CD056EC3E56E940E5002809C12BC
:0C1DC000107B12180CC2AF75EF1291CD11
:00000001FF
